:1000000019C033C032C031C030C02FC02EC02DC087
:100010002CC02BC02AC07FC028C027C026C025C046
:1000200024C023C022C021C020C01FC01EC01DC0CC
:100030001CC01BC011241FBECFEFD4E0DEBFCDBF5C
:1000400011E0A0E0B1E0EAE6FAE002C005900D920E
:10005000A432B107D9F721E0A4E2B1E001C01D92BA
:10006000A832B207E1F7E2D2FEC4CACF8FEF8AB955
:1000700087E084B980E388B9109280008AE0809399
:10008000810084EC99E09093890080938800EFE6EA
:10009000F0E0808182608083789408959DEC899F50
:1000A000912D1124969596959695E0E0F1E0928336
:1000B000990F292F220F220F920F891B81836083B2
:1000C0000895349906C0809127018F5F809327019E
:1000D00002C01092270135990AC0809126018F5FD6
:1000E0008093260190912701933368F006C0109207
:1000F000260180912701833368F01092270181E067
:10010000809325010895833328F01092260182E020
:100110008093250108951F920F920FB60F9211241C
:100120002F933F934F935F936F937F938F939F93FF
:10013000AF93BF93EF93FF9315B81BB88DE08A95EB
:10014000F1F7000081E090E00090240102C0880FE8
:10015000991F0A94E2F785B9E0912401F0E0E0509C
:10016000FF4FE081F0E0ED5FFE4F80818BB9809121
:1001700024018F5F833018F48093240102C0109211
:1001800024019FDFFF91EF91BF91AF919F918F91DC
:100190007F916F915F914F913F912F910F900FBE83
:1001A0000F901F901895E0E0F1E090E19283918329
:1001B00090832FEB35E444E0215030404040E1F79C
:1001C00000C00000813021F0823009F4E2C0C1C1DA
:1001D000E0E0F1E022E1228390E1918390835FEB04
:1001E00065E474E0515060407040E1F700C00000E9
:1001F0003CE03283918390838FEBA5E444E081500F
:10020000A0404040E1F700C0000088E08283918375
:1002100090835FEB65E474E0515060407040E1F71B
:1002200000C00000828321839083AFEB45E454E05B
:10023000A15040405040E1F700C00000828331836C
:1002400090836FEB75E4A4E061507040A040E1F74B
:1002500000C000008283818390834FEB55E464E00B
:10026000415050406040E1F700C00000828381832C
:1002700041E040837FEBA5E454E07150A040504042
:10028000E1F700C000008283818353E050836FEB6D
:1002900075E4A4E061507040A040E1F700C00000A8
:1002A0008283818380836FEB75E4A4E061507040AA
:1002B000A040E1F700C000008283818380836FEB60
:1002C00075E4A4E061507040A040E1F700C0000078
:1002D0008283818350835FEB65E474E0515060401A
:1002E0007040E1F700C00000828381834083AFEB60
:1002F00045E454E0A15040405040E1F700C0000008
:100300008283818390836FEB75E4A4E06150704039
:10031000A040E1F700C000008283318390834FEB5F
:1003200055E464E0415050406040E1F700C00000F7
:100330008283218390837FEBA5E444E07150A04049
:100340004040E1F700C000008283918390835FEB1F
:1003500065E474E0515060407040E1F700C0000077
:100360003283918390838FEBA5E434E08150A040E9
:100370003040E1F700C000002283918390834FEB6F
:1003800055E464E0415050406040E1F700C0000097
:10039000E0C0E0E0F1E022E1228380E1818380831C
:1003A0007FEB95E4A4E071509040A040E1F700C0DD
:1003B00000003CE03283818380834FEB55E464E0AE
:1003C000415050406040E1F700C0000098E0928347
:1003D000818380837FEBA5E444E07150A0404040DE
:1003E000E1F700C000009283218380835FEB65E426
:1003F00074E0515060407040E1F700C0000092830B
:1004000031838083AFEB45E454E0A150404050403D
:10041000E1F700C000009283918380836FEB75E465
:10042000A4E061507040A040E1F700C0000092835A
:10043000918341E040835FEB65E474E0515060409C
:100440007040E1F700C000009283918353E0508335
:10045000AFEB65E474E0A15060407040E1F700C08C
:100460000000928391839083AFEB65E474E0A15028
:1004700060407040E1F700C0000052839183908398
:10048000AFEB65E474E0A15060407040E1F700C05C
:100490000000428391839083AFEB65E474E0A15048
:1004A00060407040E1F700C0000082839183908338
:1004B000AFEB65E474E0A15060407040E1F700C02C
:1004C0000000828351839083AFEB55E464E0A15038
:1004D00050406040E1F700C0000082834183908378
:1004E0007FEBA5E444E07150A0404040E1F700C03C
:1004F00000008283818390835FEB65E474E0515058
:1005000060407040E1F700C0000082838183308347
:100510009FEBA5E434E09150A0403040E1F700C0EB
:1005200000008283818320834FEB55E464E04150D7
:1005300050406040E1F700C00000828381838083E7
:100540007FEB85E494E0715080409040E1F700C07B
:100550000000E0E0F1E080E1828381838083AFEB03
:1005600025E434E0A15020403040E1F700C0000015
:10057000089543983B9A8FE599E00197F1F700C001
:1005800000003B98EBE2F1E03197F1F700C000008A
:1005900086B1E3E3F8E03197F1F700C0000088701E
:1005A000089543983B9A96E09A95F1F700C0813000
:1005B00009F43B988BE291E00197F1F700C000004D
:1005C0003B980895CF93DF93D82FC8E08D2F81708B
:1005D000E8DFD695C150D1F7DF91CF9108954398C8
:1005E0003B9A86E08A95F1F700C03B98EDE5EA95E5
:1005F000F1F7000086B1E0EEF0E03197F1F700C0CE
:10060000000083FB882780F90895CF93DF93D8E01B
:10061000C0E0E5DF20E8829FC0011124C695C82B09
:10062000D150B9F78C2FDF91CF9108951FDDE0E015
:10063000F1E080E1828381838083AFE4B3EC1197A2
:10064000F1F700C0000093E1928381838083BFE7CC
:10065000CFE422E1B150C0402040E1F700C00000EB
:100660009283918380833FE74FE482E131504040A1
:100670008040E1F700C000009283918386E180838F
:100680009FE7AFE4B2E19150A040B040E1F700C075
:10069000000035E080E123E17CE16DE15EE196E17F
:1006A0004FE1828321837083CFEBA5E4B4E0C15096
:1006B000A040B040E1F700C00000828381836083E6
:1006C000CFEBA5E4B4E0C150A040B040E1F700C0DA
:1006D0000000828381835083CFEBA5E4B4E0C15056
:1006E000A040B040E1F700C00000828391834083C6
:1006F000CFEBA5E4B4E0C150A040B040E1F700C0AA
:100700000000928391832083CFEBA5E4B4E0C15035
:10071000A040B040E1F700C0000072839183808365
:10072000CFEBA5E4B4E0C150A040B040E1F700C079
:100730000000628381838083CFEBA5E4B4E0C150E5
:10074000A040B040E1F700C0000052838183808365
:10075000CFEBA5E4B4E0C150A040B040E1F700C049
:100760000000428321838083CFEBA5E4B4E0C15035
:10077000A040B040E1F700C00000228321839083B5
:10078000CFEBA5E4B4E0C150A040B040E1F700C019
:100790000000315009F085CFE0E0F1E080E1828394
:1007A00081838083809125018130B1F118F08230FE
:1007B000C1F1FACFDEDE8CEC05DF84E403DF0FDF6E
:1007C0008823E9F3D6DE8CECFDDE8EEBFBDE1DDF4D
:1007D000C82F1BDF682F70E0762F66276C0F711D06
:1007E000072E000C880B990B4FD020E030E040E83A
:1007F0005DE3AED01BD0862F6EE050DC80912501EA
:100800008111D0CFCFE724E83EE1C15020403040F5
:10081000E1F700C00000C6CF81E0C5DC10922501E1
:10082000C1CF82E0C0DC10922501BCCF70D088F02F
:100830009F5790F0B92F9927B751A0F0D1F0660FCC
:10084000771F881F991F1AF0BA95C9F712C0B130E7
:1008500081F077D0B1E0089574C0672F782F882792
:10086000B85F39F0B93FCCF3869577956795B39526
:10087000D9F73EF490958095709561957F4F8F4F95
:100880009F4F0895E89409C097FB3EF4909580959A
:10089000709561957F4F8F4F9F4F9923A9F0F92F46
:1008A00096E9BB279395F695879577956795B795C4
:1008B000F111F8CFFAF4BB0F11F460FF1BC06F5FAA
:1008C0007F4F8F4F9F4F16C0882311F096E911C0BC
:1008D000772321F09EE8872F762F05C0662371F0DD
:1008E00096E8862F70E060E02AF09A95660F771FF1
:1008F000881FDAF7880F9695879597F9089557FD21
:100900009058440F551F59F05F3F71F04795880F7D
:1009100097FB991F61F09F3F79F087950895121614
:1009200013061406551FF2CF4695F1DF08C01616C0
:1009300017061806991FF1CF869571056105089471
:100940000895E894BB2766277727CB0197F9089588
:100950000BD078C069D028F06ED018F0952309F03C
:100960005AC05FC01124EECFCADFA0F3959FD1F328
:10097000950F50E0551F629FF001729FBB27F00D4D
:10098000B11D639FAA27F00DB11DAA1F649F6627A2
:10099000B00DA11D661F829F2227B00DA11D621FF1
:1009A000739FB00DA11D621F839FA00D611D221FAB
:1009B000749F3327A00D611D231F849F600D211D8F
:1009C000822F762F6A2F11249F5750408AF0E1F032
:1009D00088234AF0EE0FFF1FBB1F661F771F881F7B
:1009E00091505040A9F79E3F510570F014C0AACF16
:1009F0005F3FECF3983EDCF3869577956795B79566
:100A0000F795E7959F5FC1F7FE2B880F911D96958F
:100A1000879597F9089597F99F6780E870E060E0FF
:100A200008959FEF80EC089500240A941616170687
:100A300018060906089500240A94121613061406CF
:100A400005060895092E0394000C11F4882352F032
:100A5000BB0F40F4BF2B11F460FF04C06F5F7F4FEA
:0A0A60008F4F9F4F0895F894FFCFC9
:100A6A00101010FC24BAAE66CEDEA4FEEE161EDA14
:100A7A0012ADF3000250802004081040A02C0C187C
:040A8A0058D0C00080
:00000001FF
